:02000000807608
:06000B00C2AFC28C80555B
:10001B00C0D0C0E0C28EC2AF758DFF758BFFE530CF
:10002B002401D4B4601B753000E5312401D4B460D5
:10003B0014753100E5322401D4B4240D75320080DF
:10004B000AF5308006F5318002F5320536BD000227
:10005B000537D0E0D0D0D2AFD28E320F0E000000D9
:10006B000000758A8A758CECD2AFD28C32758150B8
:10007B007F007E007D007C0075300075310075328D
:10008B0000752000753300758A8A758CEC758BFFB3
:10009B00758DFF758951D2A9D2ABD2AFD28CD28ECE
:1000AB00518F514A11BF314331895129B16C71487C
:1000BB00B15880F0BD00168530A085318030000529
:1000CB00853290805AE532312BF59080528D2EBDC2
:1000DB00030FE533540FF5F0240620D611E5F0801D
:1000EB000DBD05087400300105048002E530307049
:1000FB0002D2E7F5A0BD0307E5335480238002E568
:10010B0031307102D2E7F580BD010B20000474126F
:10011B00800674248002E532307202D2E7F5902219
:10012B0075F0126010F5F0C39412400960F230D6EE
:10013B000694068002E5F02230B14220063F2007EC
:10014B003CED603930B210300409EE24FC502EC265
:10015B0004802AC205802630050BEE24CD501E7E6E
:10016B000031CC8018300411EE24FD5010D205C2A2
:10017B00047E00D20331CC8004D2047E002230B145
:10018B0010300609EE24FC5037C2068033C20780BC
:10019B002F30070FEE24CD50277E000DBD07217D9C
:1001AB0000801D300616EE24FD5015D207C2067EC8
:1001BB00007537000DBD07087D008004D2067E0058
:1001CB0022EDB4010331EE22B4020331F122B40368
:1001DB000331FE22B40403511522B405035122222C
:1001EB00512522B20022E5322401D4B4240274003A
:1001FB00F532228533F053F080E533540F04B40D00
:10020B00047400B2F745F0F53322E5312401D4B480
:10021B0060027400F53122B20122753000223003E6
:10022B001DE537C3940A4016C2038530228531235E
:10023B0085322485202C532C0385332D51B622E592
:10024B002AB4AA07E52BB455028026752200752324
:10025B00007524007525077526017527017528057E
:10026B00752910752AAA752B55752C00752D005103
:10027B00B6852230852331852432E52C5403422068
:10028B00852D3322711574D051D4701E740051D446
:10029B007018711E711574D0D2E051D4700C782285
:1002AB00790C51ED08D9FB711E2222711574D051B6
:1002BB00D47015740051D4700F7822790CE651D498
:1002CB00700608D9F8711E22227A0820E704C2B7FB
:1002DB008002D2B77146712B23DAF0D2B771467117
:1002EB003422D2B774007A08C0E071346007D0E0D2
:1002FB00D2E0238003D0E023DAEE03F6B90104D277
:10030B00B78002C2B77146712B22C2B77146C2B613
:10031B00714622C2B77146D2B67146D2B771462228
:10032B00D2B67146C2B6714622D2B6714620B70418
:10033B00740080027401C2B67146220022BC000216
:10034B00812DBC0114C27FC27EC27DC27C7B007535
:10035B001E00751F107536000C20B40281227536F5
:10036B00007F00307D05C27D753000EF240A20B47C
:10037B00FAB507FA8FF0E5F0C394254015E5F0C305
:10038B00943F402DE5F0C3947F4034E5F0C394BF18
:10039B00403D207F09D51F047C00D27C812DC27F7C
:1003AB00C27E7B00751E000CBC07047C00D27C81D6
:1003BB002DC27FBB0002812DE51E23912E8063C2CF
:1003CB007FBB0002805CE51E23D2E0912E80533070
:1003DB007F3CBB0007C27E751E008039207E0CBBA4
:1003EB003CBCD27E751E007B00802AB139E518B566
:1003FB001B1AE519B51C15E51AB51D10B13991C8B5
:10040B00851831851932D2037C00801661A9D27F01
:10041B00BB00028002912EE536C394B440047C00ED
:10042B00D27C22BB0104F51E81C6BB0204F51E81E2
:10043B00C6BB0304F51E81C6BB0504F51E807CBB41
:10044B000604F51E8075BB0704F51E806EBB0811F4
:10045B00207E07F518751E008061F51B751E008048
:10046B005ABB0C04F51E8053BB0D04F51E804CBB10
:10047B000F04F51E8045BB1004F51E803EBB110416
:10048B00F51E8037BB1211207E07F519751E0080F3
:10049B002AF51C751E008023BB3904F51E801CBB7E
:1004AB003A11207E07F51A751E00800FF51D751E7B
:1004BB00008008BB3B05307E02D27D0B22E5335416
:1004CB000FF5F0240630D602F5F0B10DE53330E729
:1004DB0019E51925F0D4F5F0C39424400830D60360
:1004EB00C39406F5F085F0198017E519C395F05004
:1004FB0008E5192424D4C395F030D603C39406F52C
:10050B001922300128E51A6024C394034011E5F049
:10051B00601BC3940130D603C39406F5F0800EE53F
:10052B0032C394024007E51A13400280E122E5181A
:10053B002401D4B46010751800E5192401D4B42437
:10054B00097519008006F5188002F51922BC0010F8
:10055B00E531B400047C018007B430047C018000D9
:10056B0022BC000C207C04C2B08007E5301350F78E
:03057B00D2B022D9
:00000001FF
